:100000000C94460018950000189500001895000003
:10001000189500000C94ED0A189500001895000042
:10002000189500001895000018950000189500001C
:10003000189500001895000018950000189500000C
:1000400018950000189500000C948B10189500006E
:1000500018950000189500001895000018950000EC
:1000600018950000189500001895000018950000DC
:1000700018950000189500000C94B7101895000012
:100080001895000018950000189500008FEF8DBF9F
:10009000CCE9EAEB4E2E80E18EBFD0E1FFE05F2E8F
:1000A000A89584B7082E877F84BF88E1992781BDF2
:1000B00091BDEEEFFFE0A0E0B1E088278D9331978E
:1000C000E9F789E189B980E08093900088E18AB9F5
:1000D00080E08093980089E18093990088E1809383
:1000E0009A000E94100F662470913203706470931E
:1000F0003203A1E0B1E0E0EAF4E20E9482100E9443
:100100000F10AAE5B2E00E9436108AB78C7F826099
:100110008ABF789479B7706179BFA49AAC98A59A90
:10012000AD9880E080936100A09AA898A19AA998C0
:10013000A29AAA98A39AAB9889E189B980E08093A2
:10014000900088E18AB986E080939500579A89E10A
:100150008093990080E08093980086E080939D00D2
:1001600088E180939A0070919A00706870939A0069
:100170000E94F50E8CE00E94920F8FE711E00E9422
:10018000040FEEEAF4E20E9482100E94EE0EAD9A95
:10019000AC9A84EF91E00E94EB0F8FEB11E00E948C
:1001A000040FEEEBF4E20E9482100E94EE0EA39A7E
:1001B000E0E9F1E080E590E00197AB9A0E94DB0F67
:1001C000AB980E94DB0F482F492BB1F7AB98AD9845
:1001D000AC9884EF91E00E94EB0F0E94F50EEAECE0
:1001E000F4E20E9482100E94D50EA2EABFE0E2E68D
:1001F000F0E00E9489110E94CD0E0E94DC0E8FE774
:1002000011E00E94040F0E94F50EAD9A80E08093E9
:100210005902E2EDF4E20E9482100E94900E0E94C8
:10022000970E8FE711E00E94040FE6EDF4E20E94C2
:1002300082100E94EE0E84E893E00E94EB0F8FE79D
:1002400011E00E94040FEAEDF4E20E9482100E9485
:10025000EE0E84E893E00E94EB0F8FE711E00E941E
:10026000040FE0EEF4E20E9482100E94EE0E84E899
:1002700093E00E94EB0F8FE711E00E94040FE8EE7D
:10028000F4E20E9482100E94EE0E84E893E00E9445
:10029000EB0F8FE711E00E94040FE2EFF4E20E94FF
:1002A00082100E94EE0E84E893E00E94EB0F8FE72D
:1002B00011E00E94040FEEEFF4E20E9482100E940F
:1002C000EE0E84E893E00E94EB0F8FE711E00E94AE
:1002D000040FECE0F5E20E9482100E94EE0E84E82A
:1002E00093E00E94EB0FA9E5B2E08C918F5F8C93B5
:1002F00000915902023011F00C94090180E08093C2
:1003000059020E9480030E94F50E8FE711E00E94BF
:10031000040FECE1F5E20E9482100E94EE0E84E8E8
:1003200093E00E94EB0F0E94F50EE2EDF4E20E94D2
:1003300082100E94900E0E94970E88E592E00E9423
:10034000EB0FADEDB1E0BA93AA930E94440322965D
:10035000ADEDB1E0ECE2F5E20E9482100E94E11105
:1003600011F00C9495018FEB14E00E94040FADED99
:10037000B1E00E94E80E84E893E00E94EB0F0E9437
:100380008003AD98E0E3F5E20E9482100E94900E97
:100390000E94970E84EF91E00E94EB0FADEDB1E06B
:1003A000BA93AA930E94440322968DE0EDEDF1E00A
:1003B00001E00A93A2E4B2E00E94A511A2E4B2E037
:1003C000EAE3F5E20E9482100E94E11118F011F0B8
:1003D0000C94EC010C940C020E94A10DEAE5F2E0F1
:1003E000A1E0B1E00E94A0118FE711E00E94040F8C
:1003F000ECE3F5E20E9482100E94EE0E8FEB11E01A
:100400000E94040FAAE5B2E00E94E80E87EE93E096
:100410000E94EB0F0C9424028FE712E00E94040F5D
:10042000ECE4F5E20E9482100E94EE0E8FEB14E0E5
:100430000E94040FEAE5F5E20E9482100E94EE0E8F
:1004400087EE93E00E94EB0FA2E4B2E00E94361028
:100450000E948003AD9A0E94F50EE2E6F5E20E944A
:1004600082100E94EE0EE2E7F5E20E9482100E94E6
:10047000900E8DE00E949A0E0E94970E8CE291E001
:100480000E94EB0F88E290E00E94EB0FADEDB1E02F
:10049000BA93AA930E9444032296ADEDB1E0ECE238
:1004A000F5E20E9482100E94E11111F00C944202C8
:1004B0000E948003AD98ECE7F5E20E9482100E9452
:1004C000900E0E94970E82E390E00E94EB0FAD9A8F
:1004D0008FE711E00E94040FE4E8F5E20E94821029
:1004E0000E94EE0E84EF91E00E94EB0FADEDB1E0C3
:1004F000BA93AA930E9444032296EDEDF1E0A2E4A0
:10050000B2E00E94A01181E0E2E4F2E007E00A9389
:10051000A2E4B2E00E94A5118FEB11E00E94040F4B
:10052000A2E4B2E00E94E80EE5E0F0E00E94070FCE
:100530000E948003AD98E4E9F5E20E9482100E94D7
:10054000900E0E94970E82E390E00E94EB0FEEE97E
:10055000F5E20E9482100E94900E0E94970EE3E046
:10056000F0E00E94070F0E948003AC9A0E94F50EF3
:100570008FE711E00E94040FE8EAF5E20E94821082
:100580000E94EE0E8FEB11E00E94040FE8EBF5E203
:100590000E9482100E94EE0EA2EABFE0E2E6F0E0C6
:1005A0000E9489110E94E60EE5E0F0E00E94070F2C
:1005B00084EF91E00E94EB0FA39AE0E9F1E080E57F
:1005C00090E00197AB9A0E94DB0FAB980E94DB0F83
:1005D000482F492BB1F7AB98AC980E94F50EAD9817
:1005E00084EF91E00E94EB0FAD9A0E949003AD98CA
:1005F00084EF91E00E94EB0FAD9A0E943D06AD980A
:1006000084EF91E00E94EB0FAD9A0E946604AD98D2
:1006100084EF91E00E94EB0FAD9A0E94CA06AD985C
:1006200084EF91E00E94EB0FAD9A0E94FA06AD981C
:1006300084EF91E00E94EB0FAD9A0E94FF09AD9804
:1006400084EF91E00E94EB0FAD9A0E94700A0E9425
:10065000360B0E94D80BAD9884EF91E00E94EB0F0F
:10066000AD9A0E947C0CEDE0F0E0A9E6B3E07BE7F8
:100670000E94BA110E94CD09E1E0F0E00E94070F4C
:100680000C94EF02F894FFCFA881B9810E94361034
:100690000E945F0EACEDB1E08C930091DC01003064
:1006A00011F00C9455030C947D030D3011F00C9453
:1006B0005B030C947D030A3011F00C946A03A8814B
:1006C000B9818C91803011F40C9468030C947F03F1
:1006D0000C947D030091DC010F3118F011F00C94A3
:1006E00073030C947D03ACEDB1E08C91A881B981CA
:1006F0000E94520E8D9388278C930C944803089582
:1007000084E690E00E94EB0F0E945F0EACEDB1E03A
:100710008C930091DC01003011F00C948403089557
:100720000E94590EA8EAB1E08C930091A801013013
:1007300011F00C946504ADEDB1E0BA93AA930E9458
:1007400044032296EDEDF1E004E0A8E9B1E00E9457
:10075000AC11A8E9B1E0EEEBF5E20E9482100E9434
:10076000E11111F00C945F04ADEDB1E00E94DB11DA
:10077000EA2FFB2F33970FEFAEE0B1E00E94AC11F0
:10078000EEE0F1E001E0A1E1B1E00E94AC11A1E1F5
:10079000B1E0E4ECF5E20E9482100E94E11111F058
:1007A0000C94DE03ADEDB1E00E94DB11EA2FFB2FCC
:1007B00032970FEFAEE0B1E00E94AC11E1E0F0E063
:1007C0000E94070FA3E1B1E00E943610E6ECF5E2CB
:1007D0000E9482100E94900EAEE0B1E00E948A0E4C
:1007E0000E94970E8AE090E00E94EB0FADEDB1E021
:1007F000BA93AA930E94440322968AE090E00E9452
:10080000EB0FADEDB1E0BA93AA930E944403229698
:1008100086E1EDEDF1E00CE00A93A3E1B1E00E9486
:10082000A511EDEDF1E0AFE1B1E00E94A0118AE089
:1008300090E00E94EB0FADEDB1E0BA93AA930E9455
:1008400044032296EDEDF1E0AFE1B1E00E94A0118A
:10085000EFE1F1E00EE0AFE1B1E00E94AC11E0EDBC
:10086000F5E20E9482100E94900EAEE0B1E00E947C
:100870008A0E0E94970E84E690E00E94EB0FE2E75A
:10088000F5E20E9482100E94900E0E94970EAD9891
:1008900084E690E00E94EB0FAD9A84EF91E00E9415
:1008A000EB0FA9E5B2E08C918F5F8C930091590218
:1008B0000A3011F00C94470480E08093590284E6DA
:1008C00090E00E94EB0F0E9480030895AFE1B1E039
:1008D000EAEDF5E20E9482100E94E11111F00C9401
:1008E0008804EDE0F0E0A0E1BB2781E08C937BE79A
:1008F0000E94BA11A9E6B3E0EC91FF27ADE0B0E0A9
:1009000091E07BE70E94BD11AFE1B1E00E9436109B
:10091000AFE1B1E0EAE3F5E20E9482100E94E1114A
:1009200011F00C94AA04EDE0F0E0A0E1BB2780E018
:100930008C937BE70E94BA11A9E6B3E0EC91FF2704
:10094000ADE0B0E091E07BE70E94BD11AFE1B1E026
:100950000E943610AFE1B1E0ECEDF5E20E948210AA
:100960000E94E11111F00C94BA04A89AAFE1B1E031
:100970000E943610AFE1B1E0E0EEF5E20E94821095
:100980000E94E11111F00C94CA04A898AFE1B1E003
:100990000E943610AFE1B1E0E4EEF5E20E94821071
:1009A0000E94E11111F00C94DA04A99AAFE1B1E0D0
:1009B0000E943610AFE1B1E0E8EEF5E20E9482104D
:1009C0000E94E11111F00C94EA04A998AFE1B1E0A2
:1009D0000E943610AFE1B1E0ECEEF5E20E94821029
:1009E0000E94E11111F00C94FA04A99AAFE1B1E070
:1009F0000E943610AFE1B1E0E0EFF5E20E94821014
:100A00000E94E11111F00C940A05A998AFE1B1E040
:100A10000E943610AFE1B1E0E4EFF5E20E948210EF
:100A20000E94E11111F00C943A050E947D08AFE19B
:100A3000B1E00E943610A3E1B1E00E943610E2E777
:100A4000F5E20E9482100E94900E8DE00E949A0EA4
:100A50000E94970E8CE291E00E94EB0F0E948003AF
:100A60008FEB11E00E94040FE6EFF5E20E94821086
:100A70000E94EE0EAFE1B1E0ECE0F6E20E948210DF
:100A80000E94E11111F00C9474050E94700AA1E912
:100A9000B2E0EEE0F6E20E9482100E940F10E1E464
:100AA000F3E0A1E9B2E00E94520E0E94A011A1E978
:100AB000B2E00E94520EE2E1F6E20E9482100E9431
:100AC0000F100E94D408E2E7F5E20E9482100E9413
:100AD000900E8DE00E949A0E0E94970E8CE291E09B
:100AE0000E94EB0F0E948003AFE1B1E0E6E1F6E285
:100AF0000E9482100E94E11111F00C9489050E945D
:100B0000890BAEEEB3E00E94E5100E94D4080E946B
:100B10008003AFE1B1E0EAE1F6E20E9482100E94B8
:100B2000E11111F00C94DD05EDE0F0E0A9E6B3E091
:100B30007BE70E94BA11A1E9B2E0ECE1F6E20E9483
:100B400082100E940F10E2E4F2E0A1E9B2E00E94FC
:100B5000520E0E94A0118AE0A1E9B2E00E94520E5A
:100B60008D9388278C93A1E9B2E00E94520EEEE0AB
:100B7000F6E20E9482100E940F10E1E4F3E0A1E986
:100B8000B2E00E94520E0E94A011A1E9B2E00E94C0
:100B9000520EE2E1F6E20E9482100E940F108AE0FB
:100BA000A1E9B2E00E94520E8D9388278C930E9497
:100BB000D408AFE1B1E00E943610AFE1B1E0E4E269
:100BC000F6E20E9482100E94E11111F00C943C06A2
:100BD000A1E9B2E0EAE2F6E20E9482100E940F1060
:100BE000E2E4F2E0A1E9B2E00E94520E0E94A011FC
:100BF0008AE0A1E9B2E00E94520E8D9388278C937F
:100C0000A1E9B2E00E94520EE2E3F6E20E948210F5
:100C10000E940F108AE0A1E9B2E00E94520E8D936B
:100C200088278C93A1E9B2E00E94520EECE3F6E231
:100C30000E9482100E940F108AE0A1E9B2E00E9497
:100C4000520E8D9388278C93A1E9B2E00E94520E38
:100C5000EAE4F6E20E9482100E940F108AE0A1E905
:100C6000B2E00E94520E8D9388278C930E94D40884
:100C7000AFE1B1E00E9436100895E8E5F6E20E9487
:100C800082100E94900E0E94970E8AE090E00E94CF
:100C9000EB0FADEDB1E0BA93AA930E944403229604
:100CA0008AE090E00E94EB0FADEDB1E0BA93AA9319
:100CB0000E944403229686E1EDEDF1E00CE00A93F8
:100CC000A3E1B1E00E94A511EDEDF1E0AFE1B1E0EB
:100CD0000E94A011EFE1F1E004E0AFE1B1E00E9479
:100CE000AC11AFE1B1E0E2E6F6E20E9482100E94B0
:100CF000E11111F00C94AC068AE090E00E94EB0F39
:100D0000ADEDB1E0BA93AA930E9444032296EDEDB3
:100D1000F1E0AFE1B1E00E94A011EFE1F1E00EE0FF
:100D2000AFE1B1E00E94AC11AD9884E690E00E9482
:100D3000EB0FAD9A82E390E00E94EB0FA9E5B2E0E1
:100D40008C918F5F8C93009159020A3011F00C94B2
:100D5000940680E08093590284E690E00E94EB0FB5
:100D60000E9480038FEB11E00E94040FA3E1B1E029
:100D70000E94E80EE2E7F5E20E9482100E94900EC7
:100D80008DE00E949A0E0E94970E8CE291E00E94E4
:100D9000EB0F0895E8E6F6E20E9482100E94900EA2
:100DA0000E94970E84EF91E00E94EB0FADEDB1E051
:100DB000BA93AA930E944403229684EF91E00E9482
:100DC000EB0FADEDB1E0BA93AA930E9444032296D3
:100DD000EDEDF1E0A4E7B2E00E94A0118CE0E4E7C1
:100DE000F2E009E00A93A4E7B2E00E94A5110E9494
:100DF00080030895E4E1FEE00E94821080E40E94F6
:100E0000920F58E0D895802D0E94880F31965A9500
:100E1000C9F704C004150A0404040505ECE3FEE068
:100E20000E94821088E40E94920F58E0D895802D8D
:100E30000E94880F31965A95C9F704C020202020BF
:100E400020101010E4E6FEE00E94821088E60E9466
:100E5000920F58E0D895802D0E94880F31965A95B0
:100E6000C9F704C020200103070F0F0FECE8FEE0D4
:100E70000E94821080E70E94920F58E0D895802D42
:100E80000E94880F31965A95C9F704C0202020206F
:100E90002020200FE4EBFEE00E94821080E60E94FA
:100EA000920F58E0D895802D0E94880F31965A9560
:100EB000C9F704C02020202020040C0CECEDFEE03B
:100EC0000E94821088E50E94920F58E0D895802DEC
:100ED0000E94880F31965A95C9F704C0202020201F
:100EE00020200808E4E0FFE00E94821080E50E94D4
:100EF000920F58E0D895802D0E94880F31965A9510
:100F0000C9F704C020202020202020088FE71FE000
:100F10000E94040F80E00E94880FE2E7F6E20E9440
:100F200082100E94900E0E94970E84EF91E00E9422
:100F3000EB0FADEDB1E0BA93AA930E944403229661
:100F4000EDEDF1E0A9E8B2E00E94A01187E0E9E848
:100F5000F2E002E00A93A9E8B2E00E94A511A9E834
:100F6000B2E00E945A11A0E9B2E00C930091900205
:100F7000003080E010F009F081E08F930091900242
:100F8000043081E008F080E09F918923882311F4E8
:100F90000C94DD078FE710E10E94040FEAE7F6E208
:100FA0000E9482100E94EE0E8FE710E10E94040F53
:100FB00082E00E94880F0C94760800919002043021
:100FC00080E010F009F081E08F93009190020930E9
:100FD00081E008F080E09F918923882311F40C942C
:100FE00004088FE710E10E94040FEAE7F6E20E948E
:100FF00082100E94EE0E8FE710E10E94040F83E042
:101000000E94880F0C94760800919002093080E0CD
:1010100010F009F081E08F93009190020F3081E091
:1010200008F080E09F918923882311F40C942B0809
:101030008FE710E10E94040FEAE7F6E20E948210B7
:101040000E94EE0E8FE710E10E94040F84E00E94E0
:10105000880F0C947608009190020F3080E010F019
:1010600009F081E08F9300919002003281E008F056
:1010700080E09F918923882311F40C9452088FE714
:1010800010E10E94040FEAE7F6E20E9482100E943B
:10109000EE0E8FE710E10E94040F85E00E94880F9A
:1010A0000C94760800919002003081E009F080E015
:1010B0008F9300919002033681E009F080E09F91C8
:1010C000892B882311F40C9476088FE710E10E9495
:1010D000040FEAE7F6E20E9482100E94EE0E8FE70C
:1010E00010E10E94040F86E00E94880FE3E0F0E028
:1010F0000E94070F0E9480030895AD9A8FEB11E0C4
:101100000E94040FE6EFF5E20E9482100E94EE0EAC
:101110008FEB11E00E94040FECE7F6E20E948210D0
:101120000E94EE0EECE8F6E20E9482100E94900E01
:101130000E94970EADEDB1E0BA93AA930E944403CA
:101140002296ADEDB1E0BA93AA930E944403229691
:10115000ADEDB1E0BA93AA930E944403229687E0D2
:10116000EDEDF1E00AE10A93A1E9B2E00E94A511D8
:1011700084EF91E00E94EB0F8FEB11E00E94040FCF
:10118000A1E9B2E00E94E80E0E94D4080E94800308
:10119000E2E7F5E20E9482100E94900E0E94970EF4
:1011A0000E948003AD980895E6E9F6E20E9482105D
:1011B0000E94900E82E20E949A0EA1E0B1E00E948D
:1011C0008A0E82E20E949A0E8DE00E949A0E0E9480
:1011D000970E88EC90E00E94EB0FA1E9B2E00E942C
:1011E0008A0E8AE10E949A0E0E94970E8AE10E945E
:1011F0009A0EE1E0F0E00E94070F8DE00E949A0E47
:101200000E94970EAD9A8CE291E00E94EB0FAD9890
:1012100082E390E00E94EB0FA9E5B2E08C918F5F32
:101220008C9300915902053011F00C94020980E072
:10123000809359020895E0EAF6E20E9482100E942B
:10124000900EA1E0B1E00E948A0EE4EAF6E20E946C
:1012500082100E94900E0E94970E84E690E00E94F9
:10126000EB0F8FEB11E00E94040FE6EFF5E20E9416
:1012700082100E94EE0E8FEB11E00E94040FE6EA4E
:10128000F6E20E9482100E94EE0EEFE0F0E00E9473
:10129000070F8FEB11E00E94040FE6EFF5E20E94CA
:1012A00082100E94EE0E8FEB11E00E94040FA1E06D
:1012B000B1E00E94E80EE4E1F0E00E94070F0E9416
:1012C00080038FEB11E00E94040FE6EFF5E20E942D
:1012D00082100E94EE0EE0EBF6E20E9482100E9465
:1012E000900E0E94970E0895E0EAF6E20E948210A6
:1012F0000E94900EA7E6B2E00E948A0EE4EAF6E2AF
:101300000E9482100E94900E0E94970E84E690E048
:101310000E94EB0F8FEB11E00E94040FE6EFF5E265
:101320000E9482100E94EE0E8FEB11E00E94040FCB
:10133000E6EAF6E20E9482100E94EE0EEFE0F0E094
:101340000E94070F8FEB11E00E94040FE6EFF5E219
:101350000E9482100E94EE0E8FEB11E00E94040F9B
:10136000A1E0B1E00E94E80EE4E1F0E00E94070F86
:101370000E9480038FEB11E00E94040FE6EFF5E27C
:101380000E9482100E94EE0EE0EBF6E20E948210B4
:101390000E94900E0E94970E0895009B0C94F709EE
:1013A0008FEB11E00E94040FE6EFF5E20E9482103D
:1013B0000E94EE0E8FEB11E00E94040FE4EBF6E2C8
:1013C0000E9482100E94EE0EA7E5B2E0EAEDF5E27F
:1013D0000E9482100E940F10AC9AE1E0F0E00E949F
:1013E000070F0E941B09E4E1F0E00E94070F0E9432
:1013F00080038AE090E00E94EB0FAC980895809102
:10140000390380933E030E94FA1110ED0E941212DC
:1014100010E00E9412120E94FA1111ED0E941212A5
:101420000E943112A7E3B3E01C930E943112A8E39B
:10143000B3E01C930E943112A9E3B3E01C930E9415
:101440003112AAE3B3E01C930E943112ABE3B3E084
:101450001C930E943112ACE3B3E01C930E942F1244
:10146000ADE3B3E01C930E940912A7E3B3E09C91A3
:101470000E94D10FA7E3B3E08C93A8E3B3E09C9163
:101480000E94D10FA8E3B3E08C93A9E3B3E09C9151
:101490000E94D10FA9E3B3E08C93AAE3B3E09C913F
:1014A0000E94D10FAAE3B3E08C93ABE3B3E09C912D
:1014B0000E94D10FABE3B3E08C93ACE3B3E09C911B
:1014C0000E94D10FACE3B3E08C93ADE3B3E09C9109
:1014D0000E94D10FADE3B3E08C930E948003089586
:1014E0000E94FA1110E90E94121210E00E941212DA
:1014F0000E94FA1111E90E9412120E943112A8E40E
:10150000B3E01C930E942F12A9E4B3E01C930E9445
:101510000912A8E4B3E09C91A9E4B3E08C91AFE395
:10152000B3E08D939C9300914803003810F00C9425
:10153000A00A95E0AFE3B3E00E9415100C94BA0A3C
:10154000AFE3B3E042E00E94030E95E0AFE3B3E007
:101550000E941510AFE3B3E00E940B0EAFE3B3E0BF
:101560000D911C914FEF5FEF0E940510AFE3B3E0C8
:101570000D931C93AFE3B3E00D911C914AE050E052
:101580000E940510AFE3B3E00D931C93AFE3B3E00B
:101590000D911C9148E050E00E94180EAFE3B3E0BB
:1015A0004D935C93A1E4B3E0EFE3F3E00E940911F3
:1015B000E1E4F3E0A2EABFE00E94A011E2EAFFE06A
:1015C000A1E4B3E0112721E002E031E00E943E10E7
:1015D000E5E0F0E00E94070F08950F921F922F920E
:1015E0003F924F925F927F92AF92BF920F931F9361
:1015F0002F933F934F935F936F937F938F939F931B
:10160000AF93BF93CF93DF93EF93FF938FB78F93F6
:101610008BB78F9388278BBF0E94FA1111E40E9429
:1016200012120E942F12AAE4B3E01C930E94091226
:101630008F918BBF8F918FBFFF91EF91DF91CF91F2
:10164000BF91AF919F918F917F916F915F914F91DA
:101650003F912F911F910F91BF90AF907F905F901E
:101660004F903F902F901F900F9018958FE711E0AB
:101670000E94040FA2EABFE0E9E3F3E00E94101128
:101680000E94E60EE0ECF6E20E9482100E94EE0E4E
:10169000A2EABFE0E8E3F3E00E9410110E94E60E28
:1016A000EAE7F6E20E9482100E94EE0E8FE716E053
:1016B0000E94040FA4E7B2E00E94E80E8FEB11E055
:1016C0000E94040FE2ECF6E20E9482100E94EE0EED
:1016D000A1E4B3E00E94E80EE6ECF6E20E9482107C
:1016E0000E94EE0E8FEB19E00E94040FEAECF6E286
:1016F0000E9482100E94EE0EA2EABFE0E2E6F0E055
:101700000E9489110E94E60EE5E0F0E00E94070FBA
:101710000895A1EFB3E0E8E9F4E20E9482100E948C
:101720002E100E949E0E082F013011F00C94D60B43
:1017300081E080934D0300914D03053018F011F0C6
:101740000C94B90B0E94A40EADE4B3E0AD90BB24A1
:10175000A7E5B3E0AA0DBB1D8C9381E090E00E9449
:10176000EB0FADE4B3E08C918F5F8C9310F40C948D
:101770009B0BAEEEB3E00E94E510009158030531DB
:1017800081E009F080E08F93009158030F3F81E0E2
:1017900009F080E09F91892B882311F40C94D60BDB
:1017A00000915903013011F00C94D60B089508955F
:1017B0000895EEECF6E20E9482100E94900E0E94C4
:1017C000970EADEDB1E0BA93AA930E94440322961E
:1017D00086E60E94FF0F81E0EDEDF1E005E00A935F
:1017E000A981BA810E94A511A881B981E8EDF6E22C
:1017F0000E9482100E94E1110FB686E6481A80E02E
:10180000580A22960FBE11F00C94480C86E60E94EE
:10181000FF0F8DE0EDEDF1E001E00A93A981BA81BF
:101820000E94A511A881B981EAE3F5E20E94821025
:101830000E94E1110FB686E6481A80E0580A229607
:101840000FBE11F40C942D0C8DE0EDEDF1E001E0F4
:101850000A93AEE0B1E00E94A511E0EDF5E20E942E
:1018600082100E94900EAEE0B1E00E948A0E0E94AB
:10187000970E84E690E00E94EB0FAEE0B1E0EAE361
:10188000F5E20E9482100E94E11111F00C94D90B34
:1018900086E60E94FF0F81E0EDEDF1E002E00A93A1
:1018A000A981BA810E94A511A881B981ECE2F5E273
:1018B0000E9482100E94E1110FB686E6481A80E06D
:1018C000580A22960FBE11F00C946E0CAEE0B1E0F7
:1018D000EAE3F5E20E9482100E940F10E2E7F5E2CF
:1018E0000E9482100E94900E8DE00E949A0E0E942B
:1018F000970E0E9480030895A1EFB3E0ECE9F4E2B3
:101900000E9482100E942E100E949E0EACE4B3E052
:101910008C9300914C03013011F00C94930CA9EAC4
:10192000B1E00E9436100E94A40EABE4B3E08C93A9
:1019300000914B03003011F00C94A00C0C94C80CD7
:101940000D3011F00C94A60C0C94C80C0A3011F058
:101950000C94B50CA9EAB1E08C91803011F40C9490
:10196000B30C0C94CA0C0C94C80C00914B030F31AF
:1019700018F011F00C94BE0C0C94C80CACEDB1E056
:101980008C91A9EAB1E00E94520E8D9388278C9326
:101990000C94930C8FEB11E00E94040FEEEDF6E235
:1019A0000E9482100E94EE0EE2E0F0E00E94070F1B
:1019B0008FEB11E00E94040FA2EABFE0EBE4F3E03A
:1019C0000E9410110E94E60EE2E0F0E00E94070F74
:1019D000AEEEB3E00E94E51000914B03013011F030
:1019E0000C941A0DE2ECF6E20E9482100E94D50ED1
:1019F000A1E4B3E00E94CF0EE6ECF6E20E94821072
:101A00000E94D50E8DE00E94DF0EE6EEF6E20E9407
:101A100082100E94D50EA2EABFE0E9E6F3E00E9440
:101A200010110E94CD0E8DE00E94DF0E0E94DC0E90
:101A30000C942A0D033011F00C94220D0E947D08A5
:101A40000C942A0D88E4482F041711F00C942A0DE9
:101A50000E942B0D08950E94300D0E946F0D089575
:101A6000AAE3B3E08C910E94CA0FAAE3B3E08C937F
:101A7000ABE3B3E08C910E94CA0FABE3B3E08C936D
:101A8000ACE3B3E08C910E94CA0FACE3B3E08C935B
:101A9000ADE3B3E08C910E94CA0FADE3B3E08C9349
:101AA0000E94FA1110ED0E94121213E00E9412120D
:101AB0000E943112AAE3B3E01C930E943112ABE3FF
:101AC000B3E01C930E943112ACE3B3E01C930E947C
:101AD0002F12ADE3B3E01C930E9409120895A7E30F
:101AE000B3E08C910E94CA0FA7E3B3E08C93A8E304
:101AF000B3E08C910E94CA0FA8E3B3E08C93A9E3F2
:101B0000B3E08C910E94CA0FA9E3B3E08C930E94CA
:101B1000FA1110ED0E94121210E00E9412120E949F
:101B20003112A7E3B3E01C930E943112A8E3B3E0A3
:101B30001C930E943112A9E3B3E01C930E94091286
:101B40000895E0EFF6E20E9482100E94900E0E943B
:101B5000970EADEDB1E0BA93AA930E94440322968A
:101B6000EDEDF1E0AAE5B2E00E94A0118BE0EAE51C
:101B7000F2E00CE00A93AAE5B2E00E94A5118FE71B
:101B800011E00E94040FAAE5B2E00E94E80EE2E034
:101B9000F0E00E94070FEAEFF6E20E9482100E9436
:101BA000900E0E94970EADEDB1E0BA93AA930E94F9
:101BB00044032296EDEDF1E0A7E6B2E00E94A01109
:101BC0008BE0E7E6F2E00CE00A93A7E6B2E00E94C1
:101BD000A5118FEB11E00E94040FA7E6B2E00E946E
:101BE000E80EE2E0F0E00E94070F0E9480030895F3
:101BF000AAE6B3E0EC91FF27AEE0B0E095E07BE72A
:101C00000E94BD110895EA2FFB2F8D91809581933D
:101C10004A95D9F70895ED91FC91EF5FFF4FFC9342
:101C2000EE93089509D00E94051000FC10D008958D
:101C300003D01ED001F8F9CF0024E89457FF02C06A
:101C400009D0689400F80BD010F80124089502D050
:101C500009D00895509540954F5F5F4F0895E894DF
:101C600017FF0895009510950F5F1F4F6894089512
:101C7000352F242FE894452B11F468940895512FA3
:101C8000402F0027112780E1440F551F001F111F0F
:101C9000021B130B416018F4020F131F4E7F8A952D
:101CA00099F708958F938D918823E9F711978F9174
:101CB00008958091AD03882309F081E00895809113
:101CC000AD03882309F408950F929F93AF93BF93B8
:101CD0007F938091AD038823E1F3F8948091AD0365
:101CE0008A958093AD039091AB03ABE6B3E0A90F67
:101CF0000024B01D8C919395903409F4992790930A
:101D0000AB0378947F91BF91AF919F910F9008950D
:101D1000A2EABFE08D91882311F00CD0FBCF08958B
:101D20000E942010802D11F005D0FACF08958DE08B
:101D300001D08AE05D9BFECF8CB908958091F003BD
:101D4000882309F081E008958091F003882309F445
:101D500008957F930F929F93AF93BF938091F00369
:101D60008823E1F3F8948091F0038A958093F0033F
:101D70009091EE03AEEAB3E0A90F0024B01D8C9160
:101D80009395903409F499279093EE037894BF913A
:101D9000AF919F910F907F910895A2EABFE08D913E
:101DA000882311F00CD0FBCF08950E942010802DC5
:101DB00011F005D0FACF08958DE001D08AE00090AF
:101DC0009B0005FEFCCF80939C000895A2EABFE033
:101DD0008D91882311F09CD0FBCF08950E94201094
:101DE000802D11F095D0FACF089581E09BD015D0C9
:101DF00080E898C08FE7213039F08FEB223021F056
:101E00008FE8233009F08FEC810F0C94920F88EE4D
:101E100093E0E1D03197D9F7089583E09927DBC0AB
:101E20008AEF90E00E94EB0F8F9A8E9A8D9A8C9A8F
:101E300070916400716070936400709164007260CE
:101E400070936400709165007D7F7093650085E0FC
:101E500090E00E94EB0F709165007E7F70936500AB
:101E600097989698959A949A70916500716070937E
:101E70006500EF93FF93E4ECF0E00E94D80FFF9130
:101E8000EF91709165007E7F70936500A1D0709195
:101E90006500716070936500EF93FF93E4ECF0E0F0
:101EA0000E94D80FFF91EF91709165007E7F709333
:101EB00065008ED070916500716070936500EF933E
:101EC000FF93E4ECF0E00E94D80FFF91EF91709146
:101ED00065007E7F709365007BD09498709165005B
:101EE000716070936500EF93FF93E4ECF0E00E9463
:101EF000D80FFF91EF91709165007E7F7093650020
:101F000067D088E20FD08EE00DD086E00BD0089528
:101F100070916500726070936500829509D008D059
:101F200057D00895709165007D7F70936500F5CF5F
:101F3000859510F4949A01C09498859510F4959A1B
:101F400001C09598859510F4969A01C0969885954C
:101F500010F4979A01C09798709165007160709322
:101F60006500EF93FF93E4ECF0E00E94D80FFF913F
:101F7000EF91709165007E7F709365000895982FB2
:101F800082958F70805D8D939F70905D9D93882763
:101F90008C9308954AE0082F0E94CB110295802B64
:101FA0000895892F8F70905110F0865FFCCF0895AF
:101FB0003197F1F70895AE2FBF2F11974A2F4B2B72
:101FC000E1F70895689462F80895E89462F8089536
:101FD00081E090E000C0EF93FF93EE27E82BE92B20
:101FE00031F0E0EDF7E03197F1F70197D1F7FF918C
:101FF000EF9108955A924A92480E591E08955A92A6
:102000004A92480E8827581E08950F92B801469F9D
:102010008001479F100D569F100D0F9008950E944C
:1020200020100D920020D9F70895903041F00D91C5
:102030001C91169507959A95E1F71C930E930895B8
:10204000D895319628F48F938BB783958BBF8F915A
:102050000020089591E005C092E003C094E001C023
:1020600098E0EEDF0D929A95E1F7089582E001C0C5
:1020700084E099279D938A95E9F708952E2E3F2EA7
:10208000992781918D3209F093958823D1F79A95FC
:10209000E22DF32D112361F0091718F011F0101B38
:1020A00001C0191B28F021F080E28D931A95E9F701
:1020B00080818D3219F48D93319604C0222311F062
:1020C0008BE28D93091738F031F0091B21F080E382
:1020D0008D930A95E9F781918D938823E1F7332356
:1020E00051F0EA2FFB2F319633958E9182933A95DA
:1020F000E1F78EE28C9308950F9301E00BBF0F91EF
:10210000889408950F930027F9CF0F9302E0F6CF3C
:102110000F9303E0F3CF7F930F93AF93BF938F930E
:102120009F938FB78F938091AD0300E4081B21F438
:102130009CB10E94E20F12C00091AC03ABE6B3E089
:1021400077279CB1A00FB71F9C9383958093AD0315
:102150000395003409F400270093AC038F918FBFDF
:102160009F918F91BF91AF910F917F9118957F9320
:102170000F93AF93BF938F939F938FB78F9380915C
:10218000F00300E4081B29F490919C000E94E20FE8
:1021900013C00091EF03AEEAB3E0772790919C0063
:1021A000A00FB71F9C9383958093F0030395003491
:1021B00009F400270093EF038F918FBF9F918F91B8
:1021C000BF91AF910F917F9118956FB7F8948827C1
:1021D00093E08D939A95E9F76FBF0895040F151F4B
:1021E000261F371F0895000F111F221F331F089548
:1021F00000951095209530950F5F1F4F2F4F3F4F43
:102200000895019110810EC00191119121913081A9
:102210000BC00191108117FF05C03FEF2FEF04C0E5
:10222000008111272227332737FF03C0E1DF8DE22A
:102230008D93CF93DF93CF92DF92EF92AA24BB24AA
:10224000CC24DD24EE2440E2CAE0DD2755E093E310
:102250008881890F87FD9F7083FD907F891B8993FB
:102260005A95A9F7C0DFAA1CBB1CCC1CDD1CEE1CB8
:102270004A9551F7E894EFE0FF2782910ED0EB30BA
:10228000E0F71EF068948A2D0CD088278D93EF908C
:10229000DF90CF90DF91CF910895982F829501D054
:1022A000892F8F70805D26F0803309F4089568943B
:1022B0008D93089500271127222733271DD08A33B5
:1022C00028F4803318F005D015D0F9CF0EF490CF54
:1022D000089580538F93402F512F622F732F83DFE8
:1022E00082DF7CDF80DF8F919927080F191F291F5C
:1022F000391F08958D910895E894FCDF8032E9F349
:102300008B32D9F38930C9F38D3211F46894F2CF4E
:10231000089541E003C042E001C044E0E40F882793
:10232000F81F829138E098E1880F991F9D933A95A4
:10233000D1F74A95B1F70C949D1188278D93089594
:1023400081918D938823E1F70895099191919923C3
:1023500051F08A95D9F7319781918D930A9519F0AB
:102360008823D1F70895E9CFE199FECFEEBBFFBBFB
:102370003196089591E001C092E07B3751F47FB728
:10238000F894F2DF8D918DBBE29AE19A9A95C9F7A4
:102390007FBF77270895FF93881BF9E0001FFA9508
:1023A00011F4FF910895881F841B18F4840F8894FA
:1023B000F5CF0894F3CF8FEF83959D919923E1F7A3
:1023C0000895689401C0E894AF93BF938D9116F07F
:1023D000919103C00E942010902D891718F011F4DC
:1023E0008823A1F7BF91AF9108959198909889980B
:1023F00088980895889A899803D0889801D0899AF6
:10240000EF93FF93E6E0F0E00E94D80FFF91EF9189
:102410000895889A899AF4DF8898809BFECFF0DF30
:102420008998EECF0894111F01C0110F69F0889AA6
:1024300018F40000899802C0899A00C0E1DF8898EA
:10244000809BFECFDDDFF1CF889A8998D9DF88980D
:10245000809BFECFE8948199689462F8D1CF08946C
:1024600001C08894331F11E0889A8998C9DF889841
:10247000809BFECFC5DF889481990894111FA0F737
:10248000889A379510F4899801C0899AB9DF88989D
:10249000809BFECFB5DF089510270000E803000001
:1024A0002B37393032333433303337330000202088
:1024B000202047534D5F313238202020200020203B
:1024C00020204F4B20202020000047534D31323830
:1024D0002000415400002323200023232323200035
:1024E00023232323232320002323232323232323E2
:1024F00020002323232323232323232320002323F8
:1025000023232323232323232323200023232323C1
:1025100023232323232323232323200047534D2D29
:10252000636F65E3B8BD65BDB86500004F4B000043
:1025300041542B435042533F00003000484F4D451B
:1025400050205445A745AA4F484100004845542013
:102550005445A745AA4F48412000E0A7B120434D6C
:102560004300A9E361BB65BDB86520534D532020EE
:10257000000041542B434D47443D310041542B430F
:10258000474D4D005349454D454E532020202020B6
:102590002020200041542B434D47463D31004154FB
:1025A0002B434C49503D310020506F7274204461E0
:1025B000746120536574200044203D2000002B43AB
:1025C0004D5400002C0041542B434D47523D000018
:1025D00041542B434D47443D000031007230000010
:1025E000723100006B3000006B3100007130000070
:1025F00071310000330020202020202020202020C6
:102600002020202020202020202000003400543DC5
:10261000200043202000323100003F0047534D315D
:102620003238000068746C70000047534D31323806
:102630002D00332042616C616E732000342054659C
:102640006D7065726174657261003F20536F7374C1
:102650006F6A6E696520000041542B434D47523D1F
:1026600031002B434D47000041542B434F50533F03
:10267000000041542B43535100002000A461BE7060
:102680006F6320B261BB61BD6361000041544423AC
:10269000313032233B0041542B434D47533D000022
:1026A000415444003B00C7E2EEEDE8EC20EDE000D1
:1026B0004154480044617468696B2E203120200029
:1026C0003A00543D000043200000443D00004154C6
:1026D0002B43504D533F00002B43504D530020528D
:1026E0005334383520004F5850414E41202D2000A2
:1026F00041542B435042523D310041542B435042F0
:04270000523D320014
:00000001FF
